:020000040000FA
:101C80000E308A00492E0E308A0006193B2E061DA2
:101C9000472E903098008316263098006400033059
:101CA00081000317830118121A081A080310B426BA
:101CB0008101B42601088400040C00000000031C0C
:101CC000FF3E831699008312181620308400CA271D
:101CD0000F3A031D522E0F30C127CA270F3A03199E
:101CE0006B2E0008043A03197C2E0008053A031DE8
:101CF0007A2ECA27840A6D2E83160403A300A30339
:101D000020308400A001A1010008BB26840A040839
:101D10002302031D842E20080002031D522E840A74
:101D200021080002031D522EA001A10183122208E6
:101D300084002108831203178D0004088F002630C9
:101D4000840083010A3020020318522E20088207E3
:101D5000D82EE12E032F1D2F492F7D2F912FA32F3A
:101D600000000E308A003B2E64000619B52E061DB9
:101D7000B72E080083162106A2002008A100220821
:101D8000A000200E0F39A006200EF039A106A00EEB
:101D90000310200D0318013EA106E039A106A00E94
:101DA000A0060800C00101030102400E00003B0034
:101DB0000630A500A60183120317D2308D000E3025
:101DC0008F00F626B027BB260408B027BB26831257
:101DD00003178D0A03198F0A83010130A502031C22
:101DE000A60326082504031DE12EA62F831603173C
:101DF0008C170C1400000000831203170E088400D7
:101E00000C0883010800F626BA260408BB268312B4
:101E100003178D0A03198F0A0D081F39031D032F9D
:101E2000AB2783010130A502031CA6032608250465
:101E3000031D032FA72F402E402E831203170F30B0
:101E40008F05E0308D050E300F02403003190D0272
:101E5000031C372F10300F02003003190D02031836
:101E6000372F831603178C013C2F402E402E8316EC
:101E7000031794308C00D4278312031720308D026F
:101E8000031C8F0383120313A50B1D2FA32F402EBA
:101E9000402E831203170F308F05FC308D050E3056
:101EA0000F02403003190D02031C632F10300F0284
:101EB000003003190D020318632F831603178C01DA
:101EC000672F402E402E8316031784308C00831218
:101ED00003170008840A8C000008840A8E00D327A8
:101EE000831203178D0A03198F0A03300D05031D92
:101EF000672F0313A50B492FA32F831603178C01FC
:101F00000C140C18812F831203170C08831203176B
:101F10008D0A03198F0AB027BB268301A50B7D2FDD
:101F2000A62F840A0008831203178C00831604303E
:101F30008C00D4278C189A2F831203178D0A031351
:101F4000A50B912FA32F2008B027BB26AB27830119
:101F50000430C127632E831603132008B0272108FD
:101F600083160313A3000F3A0319BE2F2308043A64
:101F70000319BE2F2308053A031DC02F0530C127C2
:101F80002308831264000C1EC32F831203139900CD
:101F900083160800830164008C1ECC2F1A08800071
:101FA0000800402E402E8316640055308D00AA3064
:0A1FB0008D008C14000000000800F2
:02400E00693F08
:02401000FF3F70
:00000001FF
